:020000040000FA
:100000008A012F2800280028F0000308F10083123D
:100010008C1C1D289E30061CAF30910076087302A0
:1000200003198615760874020319061676087502F8
:1000300003198616F60A8C102A280C1F2A28F601A6
:100040009E30061CAF3091008611061286129F0862
:100050000C132A2871088300F00E700E0900031398
:1000600083121F21402136212C213B210B178B1796
:10007000861B3828B320031C382801307A02031D60
:10008000692801307D020319EC2804307D02031930
:10009000F22802307D020319FD2805307D02031984
:1000A000032903307D0203190E2906307D0203194E
:1000B000142921307D0203199C2820307D02031968
:1000C000A42811307D0203196E2810307D02031917
:1000D00089280C307D02031948293828D220861B34
:1000E0006F28B320031C6F280A307D0203183828BC
:1000F0007D087D077D07F7007308F8006C21F70A7B
:100100007408F8006C21F70A7508F8006C21D220F9
:100110003828D220861B8A28B320031C8A280A305C
:100120007D02031838287D08F900F8001E30F7001A
:100130006C215F21D2203828F903FF307902031D9A
:10014000AB280930F900AB28F90A0A307902031DFF
:10015000AB28F901AB287908F8001E30F7006C21B4
:100160005F21D2203828E220861BD028DD20861B84
:10017000D028DD200530FE00DD20060DFC0DFE0B35
:10018000BC28E030FC04FC090630FE00DD20060D32
:10019000FD0DFE0BC628C030FD04FD090314080048
:1001A0000310080006170F30FE00DA20FE0BD528DA
:1001B000061308008F018E01E628DD308F004630DF
:1001C0008E00E628F4308F0070308E000C10101472
:1001D0000C1CE828101008008B13F3080319FA28E8
:1001E000F303FA288B13F30A21307302031DFA2854
:1001F0002030F3008B17D22038288B13F408031912
:100200000B29F4030B298B13F40A21307402031D0C
:100210000B292030F4008B17D22038288B13F508D7
:1002200003191C29F5031C298B13F50A21307502CB
:10023000031D1C292030F5008B17D2203828831687
:1002400083308600FF30850000308100E1309F0060
:10025000831205309F000800063092008C10831630
:10026000FF3092008C1483120B1708009001831644
:100270000C10831208000C1383160C17831208004D
:10028000F60186110612861206130030FA000800E5
:100290008B13FA08031D56290130FA001E30F700AF
:1002A0008221F9005F218B17D22038280030FA0014
:1002B0002030F300F400F5008B17D220382879089D
:1002C00079077907F7008221F300F70A8221F40009
:1002D000F70A8221F500080078088C1383169A002B
:1002E00077089B008B131C1555309D00AA309D008C
:1002F0009C1483128C1F7A2983169C131C118B1754
:1003000083120800770883169B001C141A08F80053
:100310008312080000280028002800280028002850
:10032000002800280028002800280028002800288D
:10033000002800280028002800280028002800287D
:10034000002800280028002800280028002800286D
:10035000002800280028002800280028002800285D
:02400E006A3F07
:10420000000000001F0000001F0000001F00000051
:1042100000001F001F0000001F0000001F00000022
:104220001F001F001F001F001F0010001F001F00A5
:0E4230001F001F001000100010001000000002
:00000001FF
